:020000001028C6
:10002000831207309F008316D33085008601831228
:1000300086019630A4008420A40B1B2805113030C3
:10004000860087202930A4008420A40B2428303087
:10005000860087200830860087200C3086008720A5
:100060000630860087200000A001A101A201A301A3
:100070008C208601051A4928A00A20080A3C031D85
:100080004828A001A10A21080A3C031D4828A10113
:100090008C2085185028A001A101A201A3018C2069
:1000A00005186128A0032008FF3C031D60280930C3
:1000B000A000A1032108FF3C031D60280930A10016
:1000C0008C20051B7028A20A22080A3C031D6F28F9
:1000D000A201A30A23080A3C031D6F28A3018C2058
:1000E000851B8128A2032208FF3C031D80280930BC
:1000F000A200A3032308FF3C031D80280930A300AE
:100100008C2039282030A600A60B842808008515ED
:100110008420851184200800051102308600872084
:100120003230A4008420A40B9228051520308600CC
:100130008720303021078600872030302007860056
:1001400087200A30A400203086008720A40BA32833
:100150003030230786008720303022078600872032
:100160000508A600D3302605D33C031DB028643013
:0A017000A4008420A40BB9280800A5
:02400E00303F41
:00000001FF
